:0200000480007A
:100000006F00C0006F20C0276F2080279300000082
:10001000130100009301000013020000930200008E
:100020001303000093030000130400009304000076
:10003000130500009305000013060000930600005E
:100040001307000093070000130800009308000046
:100050001309000093090000130A0000930A00002E
:10006000130B0000930B0000130C0000930C000016
:10007000130D0000930D0000130E0000930E0000FE
:10008000130F0000930F000097020000938202F804
:1000900073905230178100001301412DF32240F17B
:1000A0009392C2003301510073100134EF20103AD3
:1000B00017350000130505BA6F20D01583224508B7
:1000C0007390121483204500032185008321C5000D
:1000D0000322050183224501032385018323C501F2
:1000E00003240502832445028325C5020326050354
:1000F00083264503032785038327C50303280504B7
:1001000083284504032985048329C504032A05059A
:10011000832A4505032B8505832BC505032C05067E
:10012000832C4506032D8506832DC506032E050762
:10013000832E4507032F8507832FC50703258502D7
:1001400073002010731101142322110023263100A3
:1001500023284100232A5100232C6100232E710003
:1001600023208102232291022324A1022326B1020B
:100170002328C102232AD102232CE102232EF102DB
:1001800023200105232211052324210523263105DF
:1001900023284105232A5105232C6105232E7105AF
:1001A00023208107232291072324A1072326B107B7
:1001B0002328C107232AD107232CE107232EF10787
:1001C000F312011423245100F322001023205108BC
:1001D000F322101423225108F3223014232451084F
:1001E000F322201423265108130501006F20004735
:1010000000000000000000000000000000000000E0
:1010100000000000000000000000000000000000D0
:1010200000000000000000000000000000000000C0
:1010300000000000000000000000000000000000B0
:081040000000000000000000A8
:10200000B3E7C500B367F50093F73700B306C50023
:10201000638407023386C50093070500637ED502FB
:1020200003C705009385150093871700A38FE7FE6C
:10203000E398C5FE67800000E37ED5FE93070500A8
:1020400003A70500938747009385450023AEE7FE6D
:10205000E3E8D7FE6780000067800000B367C50033
:1020600093F737003306C5006380070293F5F50F39
:10207000930705006370C50493871700A38FB7FE0D
:10208000E31CF6FE6780000093F5F50F939785003B
:10209000B3E7B70093950701B3E5F500E374C5FE18
:1020A000930705009387470023AEB7FEE3ECC7FE16
:1020B000678000006780000083470500638E07008B
:1020C0009307050003C7170093871700E31C07FE5B
:1020D0003385A7406780000013050000678000007B
:1020E00083470500938515001305150003C7F5FF09
:1020F00063880700E386E7FE3385E74067800000DA
:10210000930700006FF05FFFB367B50093F73700E8
:10211000639E07021378C6FF330805016378050341
:10212000930705006F0000019387470093854500E2
:1021300063F8070183A6070003A70500E386E6FE10
:102140003385A7403306A640138507003386C500B4
:102150006F00400103C705008347F5FF9385150015
:10216000639AE70013051500E396C5FE130500000A
:10217000678000003385E740678000009307050013
:1021800003C705009387170093851500A38FE7FE0B
:10219000E31807FE6780000003470500930600026E
:1021A000930705006318D70003C71700938717002C
:1021B000E30CD7FE9306D0026300D7069306B00265
:1021C0006300D70483C607009305000063820604FA
:1021D0001305000093871700138606FD13172500CB
:1021E00083C607003305A700131515003305A600A5
:1021F000E39206FE638005023305A040678000007D
:1022000083C617009305000093871700E39206FC2E
:10221000130500006780000083C6170093051000B7
:1022200093871700E39606FA130500006FF09FFEF0
:1022300017F6FFFF130606DD032706008327460077
:102240009355F5413367F7006306070297F6FFFFE2
:10225000938646DF9307000023A0F60013080000D2
:1022600023A2060103270600832746003367F700F1
:10227000E31207FE2320A6002322B6006F00000011
:10228000130101FF1305903423261100EFF05FFACC
:10229000130101FE1306C1001307B10113039000DF
:1022A0006F008000138707009377F500B337F300C2
:1022B000B307F04093F777029376F500938707030F
:1022C000B387F6002300F7009396C5011355450028
:1022D0009307F7FF33E5A60093D54500E314E6FC2A
:1022E0000345C100230E01006302050693050600A5
:1022F00097F6FFFF938606D117F6FFFF130686D4E5
:1023000003A7060083A74600130805009385150060
:102310003367F700B70801016302070213070000E3
:102320002320E600930700002322F60003A70600FF
:1023300083A746003367F700E31207FE03C50500D5
:1023400023A0060123A21601E31C05FA13010102D2
:102350006780000037F6FFFF3307C500B7E70300CB
:102360006370F7149356C50093820640173300003C
:10237000130343C993972200B307F30003A7070091
:102380003375C5006306070293760704638C060E57
:1023900093760708639206189306F000639ED5169D
:1023A0001367070823A0E700730005126780000089
:1023B0001757000013074704832507006384051C93
:1023C00083A74500175600000326C6022320F70006
:1023D0006382C70C03A7050093972200B307F3009D
:1023E0001357C7001317A700136EF70D1366F701F5
:1023F00023A0C7017300051297570000938707E0D9
:1024000093963600B386D70083A706006392071E13
:1024100083A7050023A0F60083A74500B7050400A5
:1024200023A2F600F3A50510B707C0FFB307F50018
:10243000B716000013070500B386D70083AE070068
:1024400003AE470083A8870003A8C7002320D70155
:102450002322C7012324170123260701938707019D
:1024600013070701E39CD7FC739005109397220094
:10247000B307F30023A0C700730005120F1000007C
:10248000678000001367070423A0E70073000512AC
:10249000678000009757000023AE07F46FF09FF3AA
:1024A0001305100497150000938505C497F6FFFFE8
:1024B000938646B517F6FFFF1306C6B803A70600B6
:1024C00083A7460013030500938515003367F700C3
:1024D000B703010163020702930700002320F600FF
:1024E000130800002322060103A7060083A7460065
:1024F0003367F700E31207FE03C5050023A066005B
:1025000023A27600E31C05FA130101FF1305300036
:1025100023261100EFF0DFD11305100497150000FA
:102520009385C5C097F6FFFF9386C6AD17F6FFFFEC
:10253000130646B103A7060083A74600130E050045
:10254000938515003367F700B70E01016302070298
:10255000930700002320F600130800002322060141
:1025600003A7060083A746003367F700E31207FEC0
:1025700003C5050023A0C60123A2D601E31C05FA6A
:102580006FF09FF81305100497150000938585BE22
:1025900097F6FFFF938606A717F6FFFF130686AA96
:1025A00003A7060083A74600130F050093851500B7
:1025B0003367F700B70F01016302070293070000BA
:1025C0002320F600130800002322060103A70600BB
:1025D00083A746003367F700E31207FE03C5050033
:1025E00023A0E60123A2F601E31C05FA6FF0DFF158
:1025F0001305100497150000938545B997F6FFFF62
:10260000938646A017F6FFFF1306C6A303A706008E
:1026100083A7460013080500938515003367F7006C
:10262000B708010163020702130700002320E60038
:10263000930700002322F60003A7060083A74600A5
:102640003367F700E31207FE03C5050023A0060168
:1026500023A21601E31C05FA6FF01FEB8325C508C2
:10266000130101FB23248104232611042322910456
:1026700023202105232E3103232C4103232A510338
:10268000232861032326710323248103232291033A
:102690002320A103232EB10193078000130405001A
:1026A0006386F516930720006380F506938745FF40
:1026B000130710006376F7009307F0006392F5228A
:1026C00003258408EFF01FC91305040003248104C7
:1026D0008320C10483244104032901048329C10305
:1026E000032A8103832A4103032B0103832BC102A5
:1026F000032C8102832C4102032D0102832DC10191
:10270000130101056FD09F9B03274508937737007E
:1027100063980708EF078000731030000327070055
:1027200083A70700630AF706130510049715000036
:10273000938545B297F6FFFF9386C68C17F6FFFF89
:102740001306469003A7060083A74600130805005A
:10275000938515003367F700B7080101630207028C
:10276000130700002320E600930700002322F60051
:1027700003A7060083A746003367F700E31207FEAE
:1027800003C5050023A0060123A21601E31C05FAD8
:1027900013053000EFF0DFA913051000EFF05FA97B
:1027A000971500009385C5A81306100497F6FFFF40
:1027B0009386468517F5FFFF1305C58803A7060016
:1027C00083A74600130E0600938515003367F700B4
:1027D000B70E010163020702930700002320F500F2
:1027E000130800002322050103A7060083A7460063
:1027F0003367F700E31207FE03C6050023A0C601F6
:1028000023A2D601E31C06FA6FF09FF8032B850282
:10281000371C0000975400009384449E172D00003D
:10282000130D4D7EB70C0400975B0000938B8BBC9F
:102830006F00C00123A2870023A08B00B717000000
:10284000330CFC00B7F703006302FC1C9357CC0069
:10285000139437003386840003260600E30006FE47
:102860009387074093972700B307FD0083A70700CE
:1028700013F60704630C06122326F100F3AD0C10C7
:10288000B707C0FFB305FC003716000013050C00A6
:102890002324B100EFF05F87630005028327C100A6
:1028A0008325810093F707086382070A3716000023
:1028B00013050C00EFF0CFF43384840073900D10F7
:1028C00083A70B0023200400E39607F69757000028
:1028D000938787B223A08B0023A087006FF01FF699
:1028E00093051004171600001306869997E6FFFF5C
:1028F0009386467117E5FFFF1305C57403A706000D
:1029000083A7460013830500130616003367F700FC
:10291000B703010163020702930700002320F500BB
:10292000130800002322050103A7060083A7460021
:102930003367F700E31207FE8345060023A0660015
:1029400023A27600E39C05FA6FF09FE4930710043E
:10295000171600001306868A97E6FFFF9386866A9D
:1029600097E5FFFF9385056E138907001306160090
:10297000B70901016F004001930700001308000030
:1029800023A0F50023A2050103A7060083A74600A4
:102990003367F700E31207FE8347060023A02601F2
:1029A00023A23601E39207FC6FF09FDE9307100429
:1029B000171600001306468197E6FFFF938686648C
:1029C00097E5FFFF93850568138A07001306160035
:1029D000B70A01016F0040019307000013080000CF
:1029E00023A0F50023A2050103A7060083A7460044
:1029F0003367F700E31207FE8347060023A0460172
:102A000023A25601E39207FC6FF09FD813050B0039
:102A1000EFF01F82F32740F163920716173600008C
:102A20001306465E9357C600130101F69397A7005D
:102A3000232E1108232C8108972500009385855C9F
:102A400093E7170023A0F500B707002093D6C50031
:102A5000370700809387F70C232EF6FEB3E7E600D6
:102A600073900718F3260018639AD716130405000D
:102A70001347F7FF9307F00197020000938242018A
:102A8000F39252307310073B7390073A97D7BF7F8A
:102A90009387876B73905710F3270034B708C07F74
:102AA000B387170173900714B7B700009387071017
:102AB00073902730B7E701007390073073504030B0
:102AC0009747C07F93870754175700002326F79234
:102AD0009747C07F9387077217570000232CF79002
:102AE00037030800174700001307C751174E0000AF
:102AF000130ECE7093072002930500001303F30317
:102B0000938888001396F50193D61700B366D60014
:102B100033866700B3C7F600330817011316C600E3
:102B2000939757002320C7002322070193F707023A
:102B300013078700B3E7F60093D51500E314EEFC06
:102B400013060009930500001305010097470000D4
:102B500023A4076AEFF08FD0B70700803304F40096
:102B60001305010023228108EFD04FD58320C1092E
:102B7000032481091301010A67800000B7F79A0E48
:102B8000B70508009387F736130700009385C5FF44
:102B900037080080370500406F00C0022FA00600F4
:102BA0001316F70193D61700B366D600B3C7D70044
:102BB0009397E7013376F5001357170093870600C4
:102BC0003367E600B3F6B70013F61700B3860601C5
:102BD000E31606FC03A006006FF09FFC93051004AB
:102BE000170600001306866C97E6FFFF9386864162
:102BF00017E5FFFF1305054503A7060083A7460059
:102C000013880500130616003367F700B7080101A3
:102C100063020702130700002320E500930700006A
:102C20002322F50003A7060083A746003367F700B9
:102C3000E31207FE8345060023A0060123A2160126
:102C4000E39C05FA13053000EFF08FDE678000008B
:102C5000971000009380003B1301A00A23902000EE
:102C600003970000930EA00A93012000631ED7452E
:102C7000971000009380003937B1FFFF130101A0C6
:102C80002391200003972000B7BEFFFF938E0EA074
:102C900093013000631AD743971000009380803669
:102CA0003711EFBE130101AA2392200003A74000B1
:102CB000B71EEFBE938E0EAA930140006316D74154
:102CC000971000009380003437A1FFFF1301A1008B
:102CD0002393200003976000B7AEFFFF938EAE00F2
:102CE000930150006312D73F971000009380603229
:102CF0001301A00A239D20FE0397A0FF930EA00AB4
:102D0000930160006312D73D9710000093806030FC
:102D100037B1FFFF130101A0239E20FE0397C0FFE0
:102D2000B7BEFFFF938E0EA093017000631ED739CC
:102D3000971000009380E02D37110000130101AAC5
:102D4000239F20FE0397E0FFB71E0000938E0EAA7C
:102D500093018000631AD737971000009380602B8F
:102D600037A1FFFF1301A10023902000039700006B
:102D7000B7AEFFFF938EAE00930190006316D73578
:102D80009710000093800029375134121301816796
:102D9000138200FE2310220283920000B75E00001F
:102DA000938E8E679301A0006390D233971000003A
:102DB0009380402637310000130181099380B0FFD2
:102DC000A3932000171200001302E22483120200D2
:102DD000B73E0000938E8E099301B0006396D22F08
:102DE0009301C00013020000B7D0FFFF9380D0CD45
:102DF0001711000013010121231011000317010016
:102E0000B7DEFFFF938EDECD6310D72D13021200C5
:102E100093022000E31A52FC9301D0001302000039
:102E2000B7C0FFFF9380D0CC171100001301811DA4
:102E3000130000002311110003172100B7CEFFFF7C
:102E4000938EDECC6312D729130212009302200066
:102E5000E31852FC9301E00013020000B7C0FFFF2B
:102E60009380C0BC171100001301C11913000000AA
:102E7000130000002312110003174100B7CEFFFF1B
:102E8000938ECEBC6312D72513021200930220004A
:102E9000E31652FC9301F00013020000B7B0FFFFED
:102EA0009380C0BB130000001711000013018115AF
:102EB0002313110003176100B7BEFFFF938ECEBB33
:102EC0006314D7211302120093022000E31852FC6E
:102ED0009301000113020000B7B0FFFF9380B0AB75
:102EE00013000000171100001301C11113000000AE
:102EF0002314110003178100B7BEFFFF938EBEABF2
:102F00006314D71D1302120093022000E31652FC33
:102F10009301100113020000B7E0FFFF9380B0AAF5
:102F20001300000013000000171100001301810DB1
:102F3000231511000317A100B7EEFFFF938EBEAA61
:102F40006314D7191302120093022000E31652FCF7
:102F50009301200113020000171100001301810AE0
:102F6000B7200000938030232310110003170100C5
:102F7000B72E0000938E3E236318D715130212005C
:102F800093022000E31A52FC930130011302000067
:102F90001711000013010107B710000093803022C1
:102FA000130000002311110003172100B71E0000B9
:102FB000938E3E22631AD71113021200930220004F
:102FC000E31852FC930140011302000017110000A6
:102FD00013014103B710000093802012130000007A
:102FE000130000002312110003174100B71E000058
:102FF000938E2E12631AD70D130212009302200033
:10300000E31652FC93015001130200001711000057
:10301000130141FF1300000093002011231311003E
:1030200003176100930E20116310D70B13021200D7
:1030300093022000E31C52FC930160011302000084
:1030400017110000130101FC130000009300100190
:10305000130000002314110003178100930E1001C8
:103060006314D7071302120093022000E31A52FCE4
:10307000930170011302000017110000130181F881
:103080001300000013000000B73000009380100010
:10309000231511000317A100B73E0000938E1E00F8
:1030A0006314D7031302120093022000E31652FCAC
:1030B00037C500001305F5EE97150000938585F4DC
:1030C0002393A500631A30001395110063000500D7
:1030D0001365150073000000130510007300000055
:0430E000731000C0A9
:1030E400417373657274696F6E206661696C65649F
:1030F4003A2061646472203E3D202831554C203CC6
:103104003C203132292026262061646472203C2030
:103114003633202A202831554C203C3C203132299A
:103124000A000000417373657274696F6E206661F2
:10313400696C65643A20212870745B315D5B61645D
:1031440064722F2831554C203C3C203132295D20BB
:103154002620307830383029202626206361757384
:1031640065203D3D203078660A0000004173736598
:103174007274696F6E206661696C65643A206E6F63
:1031840064650A00417373657274696F6E206661C9
:10319400696C65643A20757365725F6D61707069FE
:1031A4006E675B616464722F2831554C203C3C206F
:1031B4003132295D2E61646472203D3D20300A0065
:1031C400417373657274696F6E206661696C6564BE
:1031D4003A2070745B315D5B616464722F283155F1
:1031E4004C203C3C203132295D202620307830347C
:1031F400300A0000417373657274696F6E206661F2
:10320400696C65643A2070745B315D5B61646472FF
:103214002F2831554C203C3C203132295D2026207A
:1032240030783038300A0000417373657274696F06
:103234006E206661696C65643A2074662D3E657023
:103244006320252034203D3D20300A0041737365FE
:103254007274696F6E206661696C65643A2021221C
:10326400696C6C6567616C20696E737472756374E4
:10327400696F6E220A000000417373657274696F8E
:103284006E206661696C65643A202122756E6578EA
:1032940070656374656420657863657074696F6EC6
:1032A400220A0000417373657274696F6E2066614F
:1032B400696C65643A202122756E737570706F7243
:1032C4007465642073617470206D6F6465220A00F4
:10400000EFBEEFBEEFBEEFBEEFBEEFBEEFBEEFBE48
:04401000EFBEEFBE52
:040000058000000077
:00000001FF
